:020000040000FA
:06000000D38C0BEF13F09E
:020006000000F8
:08000800F2B407D0A490222AF3
:080010001100F6D7F5D7F4D773
:0800180002D0F29411009E9C3D
:10002000E8CF01F1D8CF02F1E0CF03F1F6CF06F12E
:10003000F7CF07F1F5CF09F1F4CF0AF1F3CF0BF1C8
:100040000101295118272A5119232B511A2308E39A
:1000500087CF50F188CF51F122C052F11C8E5B91B5
:100060001B4E02900201C1CF73F2C1A40ED0C29008
:10007000192A030EC11407E0C350C11404E0C35091
:10008000C11401E0C350C28084D099B248D0560E4A
:100090009912C450236F0427C350226F0327D8B08E
:1000A000042B22C224F223C225F21651225F1751DB
:1000B000235B04E324C216F225C217F2C4500627BC
:1000C000C3500527D8B0062BC4500827C3500727B4
:1000D000D8B0082BC4500A27C3500927D8B00A2B20
:1000E000012F57D0400E016F03C236F204C237F21F
:1000F00005C238F206C239F207C23AF208C23BF230
:1001000009C23CF20AC23DF2036B046B056B066B3D
:10011000076B086B096B0A6B188018823AD0560E71
:10012000E81C9916C4500C27C3500B27D8B00C2BD1
:10013000C4500E27C3500D27D8B00E2BC450102723
:10014000C3500F27D8B0102BC4501227C35011270B
:10015000D8B0122B022F1DD0400E026F0BC23EF200
:100160000CC23FF20DC240F20EC241F20FC242F287
:1001700010C243F211C244F212C245F20B6B0C6B77
:100180000D6B0E6B0F6B106B116B126B188018845C
:1001900000D00101282A5F2F08D0140E5F6F292A92
:1001A000008403668C7803660306602F05D0BC0EBE
:1001B000606F2A2A00881C82612F08D0622F06D027
:1001C000540E616F080E626F2B2A0080204E1C8A2D
:1001D000D7EC0DF09EAC03D09E9C1F2A31D706C1F0
:1001E000F6FF07C1F7FF09C1F5FF0AC1F4FF0BC114
:1001F000F3FF03C1E0FF01C1E8FF02C1D8FF100017
:04020000A4981000AE
:0C0204000BEF13F00000240348066A0909
:100210008C0CAB0FC812E215F9180B1C1A1F232205
:10022000282526281F2B112EFB30DF33BA368C39B8
:10023000563C173FCE417A441C47B4493F4CBF4E11
:1002400033519B53F5554258825AB35CD75EEB60ED
:10025000F162E864CF66A6686D6A236CC96D5E6F53
:10026000E2705472B573047541766B77847889793E
:100270007C7A5C7B297CE37C897D1D7E9C7E097F6A
:10028000617FA67FD87FF57FFF7FF57FD87FA67F30
:10029000617F097F9C7E1D7E897DE37C297C5C7B60
:1002A0007C7A897984786B7741760475B57354725A
:1002B000E2705E6FC96D236C6D6AA668CF66E864F4
:1002C000F162EB60D75EB35C825A4258F5559B539E
:1002D0003351BF4E3F4CB4491C477A44CE41173F7F
:1002E000563C8C39BA36DF33FB30112E1F2B2628B3
:1002F000282523221A1F0B1CF918E215C812AB0F70
:100300008C0C6A09480624030000DCFCB8F996F658
:1003100074F355F038ED1EEA07E7F5E3E6E0DDDDBE
:10032000D8DADAD7E1D4EFD105CF21CC46C974C6EB
:10033000AAC3E9C032BE86BBE4B84CB6C1B341B172
:10034000CDAE65AC0BAABEA77EA54DA329A1159F76
:100350000F9D189B31995A979395DD933792A290F0
:100360001E8FAC8D4B8CFC8ABF8995887C877786E5
:100370008485A484D7831D837782E3816481F78099
:100380009F805A8028800B8001800B8028805A80B3
:100390009F80F7806481E38177821D83D783A48463
:1003A000848577867C879588BF89FC8A4B8CAC8D49
:1003B0001E8FA2903792DD9393955A973199189B8F
:1003C0000F9D159F29A14DA37EA5BEA70BAA65ACC5
:1003D000CDAE41B1C1B34CB6E4B886BB32BEE9C0C4
:1003E000AAC374C646C921CC05CFEFD1E1D4DAD770
:1003F000D8DADDDDE6E0F5E307E71EEA38ED55F093
:1004000074F396F6B8F9DCFC11001F002F003B00D6
:10041000490059006700710089009500A300B300EE
:10042000C100D300DF00EF00FB000D011B0125011F
:1004300039014B015B016701750185019101A30140
:10044000AF01BB01CD01DF01EB01F70109021D0284
:1004500023023302410251025F026B0281028D02CC
:10046000A102AB02BD02C502D702E702F5020503F5
:1004700013031D0335033D0355035F036D0377032A
:100480008B039703A903B903C703D703E503F1035C
:10049000FD030F041B042D043F0449045D0469049B
:1004A0007F048B049304A304B104C104CF04E104CA
:1004B000EB04FD040B051B0529052F055105570508
:1004C00065057705810593059F05AD05BF05CF053A
:1004D000DB05E705FB050706170623062F0647067B
:1004E0005306650679067F0685069D06AD06BB06A2
:1004F000CD06D906DF06F706090713071F073707DA
:1005000045074F0761076D0779078B079D079F0711
:10051000B507C907D307E107F70705080F08210842
:1005200033083F08510859086908710883089B0877
:10053000A508AD08C308CB08E108EF08F9080709CA
:100540001D092B093509490959096B0977098509DD
:100550008F09A309AD09C709C709D909EB09FD0925
:10056000130A130A210A390A490A570A630A6F0A49
:10057000810A930A9F0AAB0ABD0ACF0AD90AE70A81
:10058000F30A030B150B230B2D0B3F0B510B5D0BCC
:100590006F0B7B0B8D0B9B0BB70BB90BC30BCF0BEF
:1005A000E10BF50B070C110C250C2F0C410C410C29
:1005B0005B0C6D0C770C890C950C9D0CB50CC70C65
:1005C000C70CE30CF10C010D0F0D1F0D2B0D3D0D94
:1005D0004F0D550D690D790D850D8D0DA30DAB0DCD
:1005E000BD0DCD0DDB0DE70DFD0D090E170E270E10
:1005F000350E4B0E570E5D0E710E7D0E8F0E9B0E3F
:10060000B10EB90ED10EDB0E5D0100BD0200190462
:1006100000770500D306003308008F0900ED0A00BB
:10062000410C00AB0D00070F00691000C311001949
:100630001300751400D715003317008F1800ED193B
:10064000004F1B00A51C000B1E00671F00C52000EB
:10065000212200832300DD24003B26009B2700F796
:100660002800552A00A92B00072D006F2E00CF2F40
:10067000002731008D3200EB33004135008F36000A
:10068000F737005B3900B73A00113C00733D00C9F1
:100690003E002B4000934100E34200454400A34547
:1006A000000547005B4800B54900134B00734C0040
:1006B000D74D002D4F00935000F551004B5300A92A
:1006C00054000B5600615700C158001F5A00795B57
:1006D00000D75C00395E00955F00F5600051620054
:1006E000B363000B6500616600C167002969007B88
:1006F0006A00DB6B00396D00956E00F56F0051717B
:1007000000B372001574006B7500C3760025780085
:10071000917900ED7A00377C009F7D00FB7E004BD5
:100720008000B381000B8300778400CD85002B8788
:1007300000858800EF8900578B009F8C00018E0098
:10074000598F00B99000159200739300E194003125
:100750009600939700E398004B9A00A79B00019D99
:10076000005F9E00C19F001BA10079A200D5A300DD
:1007700035A50093A600EDA70043A900ABAA000988
:10078000AC0065AD00C5AE001BB0007FB100D3B2B8
:10079000003DB40099B500EFB60055B800ADB90002
:1007A00009BB006FBC00CDBD0033BF007FC000E1BE
:1007B000C10047C3009DC400FBC50057C700B7C8B0
:1007C0000009CA0071CB00D1CC002FCE0089CF0028
:1007D000E7D00047D200A5D300F9D4005DD600BD14
:1007E000D7001BD90077DA00CDDB0035DD0097DEBE
:1007F00000F1DF0043E100ABE20001E40067E50047
:10080000BDE6001BE8007BE900DFEA0029EC00956B
:10081000ED00F1EE004FF000AFF1000BF30063F4D8
:1008200000C9F5002DF70081F800E9F9003FFB0051
:1008300097FC00F3FD004DFF00B100011302016DB4
:100840000301CB04011F06017D0701DF0801410AF6
:10085000019B0B01FF0C01530E01B50F0117110194
:10086000691201CF13012D15017D1601DF17013F1C
:100870001901A11A01FD1B01531D01AB1E01172017
:1008800001732101D122012D24018D2501EF2601C3
:100890004D2801AF2901FF2A016B2C01BB2D011747
:1008A0002F017F3001DD31013333018D3401E93512
:1008B000014D3701A73801033A01613B01C93C01F1
:1008C0001F3E01873F01DB4001374201954301E9AB
:1008D0004401514601B347010F49016D4A01D34B11
:1008E00001314D01874E01E74F01455101955201FC
:1008F000FD5301575501BB56010F58016B5901C3F8
:100900005A01235C01855D01BD02007705003308B3
:1009100000ED0A00AB0D00691000191300D7150097
:100920008F18004F1B000B1E00C520008323003BC7
:100930002600F72800A92B006F2E00273100EB338B
:10094000008F36005B3900113C00C93E0093410026
:10095000454400054700B54900734C002D4F00F594
:100960005100A954006157001F5A00D75C00955FE1
:10097000005162000B6500C167007B6A00396D00A1
:10098000F56F00B372006B7500257800ED7A009F5B
:100990007D004B80000B8300CD8500858800578B40
:1009A00000018E00B99000739300319600E3980027
:1009B000A79B005F9E001BA100D5A30093A6004348
:1009C000A90009AC00C5AE007FB1003DB400EFB690
:1009D00000ADB9006FBC0033BF00E1C1009DC40091
:1009E00057C70009CA00D1CC0089CF0047D200F90F
:1009F000D400BDD70077DA0035DD00F1DF00ABE2CF
:100A00000067E5001BE800DFEA0095ED004FF0000D
:100A10000BF300C9F50081F8003FFB00F3FD00B1C6
:100A200000016D03011F0601DF08019B0B01530E3E
:100A300001171101CF13017D16013F1901FD1B01A3
:100A4000AB1E017321012D2401EF2601AF29016B9B
:100A50002C01172F01DD31018D34014D3701033A8F
:100A600001C93C01873F01374201E94401B3470115
:100A70006D4A01314D01E74F019552015755010F64
:100A80005801C35A01855D013D6001076301B965E5
:100A9000016D68013B6B01F36D01AB70015F730188
:100AA0001D7601D57801917B014F7E01038101BB49
:100AB00083017986013D8901F38B01AD8E01699136
:100AC00001219401E19601939901559C01159F0123
:100AD000CDA1017FA40147A701F9A901B7AC017B12
:100AE000AF012DB201E7B4019FB70151BA011BBD9F
:100AF00001D3BF018FC20149C50105C801C3CA01A5
:100B000083CD013BD001EDD201A9D50169D80125E2
:100B1000DB01D7DD0197E00155E30111E601CBE8E8
:100B2000017DEB0135EE01F3F001BBF30175F60138
:100B300021F901E5FB01A9FE01670102110402D1BF
:100B400006028F09024B0C02050F02C111027F142D
:100B500002451702F11902A71C02651F0225220295
:100B6000E92402992702532A020F2D02BB2F027F8C
:100B700032023D3502F73702B33A02713D022F408F
:100B800002E742029B45026348021B4B02CF4D0223
:100B90008D5002495302015602D958027D5B02373B
:100BA0005E02EF6002AD63026B6602276902EB6BC7
:100BB000029D6E025171020D7402BF7602A179028C
:100BC000417C02F57E02B781027B8402298702DB29
:100BD00089029F8C025B8F020F9202D99402839745
:100BE00002539A02079D02AB9F0277A2022FA50231
:100BF000F3A702ABAA0267AD0221B002D9B20291FB
:100C0000B50253B80207BB02770500ED0A00691070
:100C100000D715004F1B00C520003B2600A92B0064
:100C20002731008F3600113C0093410005470073C7
:100C30004C00F55100615700D75C00516200C1675C
:100C400000396D00B372002578009F7D000B830092
:100C5000858800018E00739300E398005F9E00D5A5
:100C6000A30043A900C5AE003DB400ADB90033BF39
:100C7000009DC40009CA0089CF00F9D40077DA00CA
:100C8000F1DF0067E500DFEA004FF000C9F5003F43
:100C9000FB00B100011F06019B0B011711017D161E
:100CA00001FD1B01732101EF26016B2C01DD3101D8
:100CB0004D3701C93C01374201B34701314D019520
:100CC00052010F5801855D010763016D6801F36DE5
:100CD000015F7301D578014F7E01BB83013D89011E
:100CE000AD8E01219401939901159F017FA401F913
:100CF000A9017BAF01E7B40151BA01D3BF0149C5D6
:100D000001C3CA013BD001A9D50125DB0197E00150
:100D100011E6017DEB01F3F00175F601E5FB0167DA
:100D20000102D106024B0C02C11102451702A71C99
:100D3000022522029927020F2D027F3202F7370285
:100D4000713D02E74202634802CF4D02495302D986
:100D50005802375E02AD63022769029D6E020D7470
:100D600002A17902F57E027B8402DB89025B8F029D
:100D7000D99402539A02AB9F022FA502ABAA02217B
:100D8000B00291B50207BB0289C002F7C5026FCB62
:100D900002E9D0025BD602D5DB0251E102C3E602D2
:100DA00031EC02A3F10213F70295FC021102038158
:100DB0000703FB0C03711203E91703651D03CF2220
:100DC00003452803BF2D03353303B938031B3E0306
:100DD0009F43030D49037F4E03FB53036F5903E504
:100DE0005E03556403D16903416F03B77403357A19
:100DF00003A37F031B8503918A031190038D950341
:100E0000FF9A0369A003E9A50359AB03D1B0033FDF
:100E1000B603BDBB0339C103A7C6031DCC0393D1E1
:100E2000030FD70387DC03FDE1036BE703E1EC036A
:100E300063F203CFF7034BFD03C502041D080495BD
:100E40000D041D13049718041B1E047F2304ED28B2
:100E500004712E04DF3304573904CB3E04434404A9
:100E6000BF49042D4F04A95404255A04955F040773
:100E70006504896A04F36F047F7504E37A0455807E
:100E800004B98504458B04BD9004319604A79B04E6
:100E90001DA10495A6040FAC047FB104FDB6046B3C
:100EA000BC04EFC1044BC704C9CC043FD204BBD778
:100EB000043DDD0499E20421E80493ED0409F30400
:100EC00079F804FBFD045F0305DF0805550E05CD29
:100ED00013054D1905B31E05212405A52905252F48
:100EE00005953405FF39057D3F05F14405614A0547
:100EF000F54F05595505DD5A05476005AF650527CE
:100F00006B059D7005197605ED0A00D71500C52003
:100F100000A92B008F3600934100734C00615700ED
:100F2000516200396D002578000B8300018E00E3CB
:100F30009800D5A300C5AE00ADB9009DC40089CF0F
:100F40000077DA0067E5004FF0003FFB001F060165
:100F5000171101FD1B01EF2601DD3101C93C01B371
:100F60004701955201855D016D68015F73014F7EF8
:100F7000013D8901219401159F01F9A901E7B401FF
:100F8000D3BF01C3CA01A9D50197E0017DEB01756B
:100F9000F6016701024B0C024517022522020F2DB4
:100FA00002F73702E74202CF4D02D95802AD630281
:100FB0009D6E02A179027B84025B8F02539A022FFD
:100FC000A50221B00207BB02F7C502E9D002D5DBBA
:100FD00002C3E602A3F10295FC028107037112032A
:100FE000651D034528033533031B3E030D4903FBF1
:100FF0005303E55E03D16903B77403A37F03918AAA
:10100000038D950369A00359AB033FB60339C103B0
:101010001DCC030FD703FDE103E1EC03CFF703C5BC
:101020000204950D049718047F2304712E04573988
:10103000044344042D4F04255A04076504F36F0448
:10104000E37A04B98504BD9004A79B0495A6047FA8
:10105000B1046BBC044BC7043FD2043DDD0421E85E
:101060000409F304FBFD04DF0805CD1305B31E05D9
:10107000A529059534057D3F05614A055955054764
:101080006005276B051976052D8105E98B05E3962B
:1010900005C9A105B9AC059FB70593C2057FCD056C
:1010A00069D80555E30541EE051DF9051F0406073E
:1010B0000F06ED1906C72406BF2F06BB3A06A14549
:1010C00006995006755B06656606577106437C06F1
:1010D0002587060B92060D9D06F9A706DFB206C707
:1010E000BD06ADC806A9D30691DE0677E90667F40A
:1010F000064DFF06450A072B15070D2007FD2A0799
:10110000EF3507D74007CD4B07AD5607A761078BD3
:101110006C077977075182074F8D0741980727A3FE
:101120000715AE0701B907EDC307D7CE07C3D90727
:10113000B7E407A7EF0787FA076D0508671008519E
:101140001B083D26082531080F3C08FD4608E951DB
:1011500008DB5C08CB6708B17208997D088B8808AA
:101160007B93085B9E084FA90835B4083FBF08135E
:10117000CA0803D508F1DF08DBEA08C1F508AD00AD
:1011800009990B097B1609732109632C0955370945
:10119000474209234D09135809F96209EB6D09D734
:1011A0007809CB8309AB8E0997990981A40975AF9A
:1011B000095BBA094DC50939D00931DB090FE609C8
:1011C000FDF009E3FB09D9060ABB110AA51C0A9D1B
:1011D000270A8F320A6F3D0A63480A47530A3F5E67
:1011E0000A25690A11740AE77E0AE5890ABD940A8C
:1011F000BD9F0AADAA0A8DB50A87C00A6DCB0A4DFC
:08120000D60A4FE10A2FEC0AA7
:081208000001A68E05B00AD01A
:1012100005B23ED005B431D005B624D029C06CF05B
:101220000586120007BE43D007A005D00BC009F009
:10123000078E07903CD007A205D00CC009F0078E9E
:10124000079235D007A405D00DC009F0078E07948A
:101250002ED007A605D00EC009F0078E079627D01E
:10126000058812006C51295C3408D8B0F10C058453
:101270008C9E280E73EC09F012006C51295C3E081C
:10128000D8B0F20C05828C9E280E73EC09F0120087
:101290006C51295C3F08D8B0F30C05808C9E280E59
:1012A00073EC09F0096A0A6A086A059A078E05BA9A
:1012B00068D0058A320EF66E220EF76EA68EF86A98
:1012C0000950330844E2079E059C059A059E656B0C
:1012D0001200F55008E106A8F6D7069815C113F1DB
:1012E00016C114F1120000018C9C756F766F753B6E
:1012F000F00E9516751376138C500F0975158C6EBC
:101300008C8A24D88C9A22D80F0976158C6E8C8AF8
:101310008C9A0F0E9512120000B4D4D98C9E0F0E29
:1013200095128C8C8C8A12D883A607D0D890774BD4
:10133000782BD8B0056A060002D0776B786B8C9A50
:1013400005D88C8A03D88C9A8C9C1200120009C094
:1013500066F0676BD890663767376651F626675137
:10136000F722A68E0900F5CF66F00900F5CFF7FF4A
:1013700066C0F6FF0900F6CF13F1F7CF14F1F5CFF1
:1013800008F005BC07D0C8DF058C0850E88E8C9E9D
:1013900073EC09F006B452D1BFDF8C8E0A5004E121
:1013A000FF0E091401E18C9E05BE59D17FD98CAE88
:1013B00090D70F0EF5648DD7200EF5608AD7100EEA
:1013C000F55C000102EC14F00FD041D04BD054D0AA
:1013D00064D0B3D0CFD0D4D00FD078D0DED00CD062
:1013E0000BD00AD009D008D0020E46D900EE6DF01D
:1013F00012C066F0E1D833D1010E656F3A0E646F0A
:10140000058E54D9F5CFE9FF04B4F5CF11F14ED9CB
:10141000F5CFEAFF04B4F5CF12F10494EECF12F049
:101420006D0E626F000E636F00EE6DF012C066F01D
:101430006651C7D8049462C0E9FF63C0EAFF654FF4
:10144000059EEE50E9CF62F0EACF63F04CD7040E70
:1014500013D900EE6DF013C066F0AED812C066F07E
:10146000ABD8FDD0020E08D9136AB1D800EE6DF0EA
:1014700067C066F0A1D8F3D0050EFED8A8D800EE5C
:101480006DF069C066F098D868C066F095D867C0FE
:1014900066F092D8624B632BE2D0040EEDD8136A4B
:1014A00012AE04D0059E121E122A129E90D800EE93
:1014B0006DF068C066F080D867C066F07DD8200EF9
:1014C0006D6F2D0E05AE6D6F058EC9D0060ED4D88A
:1014D00013AE06D0059E121E131E124A132A139E27
:1014E000686B696B12500A0DF3CF66F0F4CF67F0AA
:1014F00013500A0DF3506727F4506823040E696FE8
:10150000D890683367336633692FFAD766C012F014
:1015100067C013F05CD800EE6DF0200EEE6E68C070
:1015200066F04AD867394DD82E0EEE6E675149D80D
:101530002D0E05AE6D6F058E92D0060E9DD813AEA2
:1015400006D0059E121E131E123E132A139E3FD86C
:1015500000EE6DF069C066F02FD868C066F02CD838
:1015600067C066F029D8200E6D6F2D0E05AE6D6F29
:10157000058E75D09BD8059EF550E88E8C9EB3D60F
:101580000484048693D8F5CF7FF090D8F5CF80F00F
:1015900004987F51806504881200068887D8F5CFAB
:1015A000E9FF84D8F5CFEAFFEF50096E0A6A13C14C
:1015B00015F114C116F189D6663903D8665101D8E0
:1015C00012000F0B300F6465070FEE6E1200F29ED3
:1015D000FDCF0DF1FECF0EF1FFCF0FF10600F28E21
:1015E0000684D8900F0E6B6F010E666F676B686B89
:1015F000696B12371337673768376937664F1200E0
:1016000000EE66F0EC5007E0030FE8B6EF6EEF5027
:10161000300FE8BEEF6EEC5007E0030FE8B6EF6E58
:10162000EF50300FE8BEEF6EEC50E3E0030FE8B68A
:10163000EF6EEF50300FE8BEEF6EDBD7010E666F36
:101640006B2FDED7069405000101F29E0D51FD6E51
:101650000E51FE6E0F51FF6EF28E0001D1D7049431
:1016600062C0E9FF63C0EAFF654F059EEE50E9CF17
:1016700062F0EACF63F037D6656F18D8F5CFE9FF8F
:1016800004B4F5CF11F112D8F5CFEAFF04B4F5CFC9
:1016900012F10494EECF12F0EECF13F0058E3A0E55
:1016A000646F6D0E626F000E636F1200A68E13C121
:1016B000F6FF14C1F7FFF86A0900F6CF13F1F7CF70
:1016C00014F1120000948C9A8C8C8C9E0F0E951243
:1016D00083A4159E83B4158E83A0159C83B0158CAE
:1016E000008600A81200009883A6149E83B6148E6C
:1016F00083A4149C83B4148C83A2149A83B2148A96
:1017000083A0149883B0148883A6159883B615888F
:1017100083A2159A83B2158A8C8E8C9C83A614960C
:1017200083B6148683A4149483B4148483A214927D
:1017300083B2148283A0149083B0148083A615967C
:1017400083B6158683A4159483B4158483A2159259
:1017500083B2158283A0159083B0158015503F0B7E
:101760007A6303D081C07EF012007E2F120081C008
:101770007EF0008215503F0B7A6F1200000105A821
:101780001200A0D700010092010115A21D8215A22E
:101790001D9415A41D8215A41D8415B605D03051C5
:1017A00002E11C7801D01D8800011550200B7D63DB
:1017B00001D01AD01F0E03267D6F06B615D015BABC
:1017C00013D004B00BD004A60FD00480030E165C17
:1017D000D8B41D800001040E616F06D004901D90E6
:1017E0000001050E616F06801200120000010096D4
:1017F0001550C00BE8BEE87C7B6301D012007B6112
:1018000015D07C077F0E7C6154D0040E032606A6FB
:10181000176A800E7C6F06B62AD004B01BD00496DF
:101820001606D8B041D0100E166E3ED07C2B810E1D
:101830007C653FD0080E032606A6176A800E7C6FD3
:1018400006B61BD004B01FD00496162A110E1660DF
:10185000166A2AD0E9CF04F1EACF05F111C1E9FFF8
:1018600012C1EAFF7F5104A8EF62EF0618D0010110
:10187000000E32633207000112000101FF0E3263D5
:10188000322B000116D0E9CF04F1EACF05F111C1E6
:10189000E9FF12C1EAFF805104A8EF62EF2A04C1F8
:1018A000E9FF05C1EAFF00D01650150F0D6E05982F
:1018B00007841550C00BE8BEE87C7B6F1200120055
:1018C00001011C923051030D3C513EE0E84C41D0E7
:1018D000E84C44D0E84C47D03CC1F6FFF76AF636F6
:1018E000F736F690F86A080EF626040EF722000E78
:1018F000F8220900F5503003F3CF3DF1F4CF3EF16B
:101900003F6B0900F5503003F3503E27F4503F235E
:10191000F29C3DC129F13EC12AF13FC12BF1F28C6D
:10192000435130033F6B44313F33E8303F333F0B8B
:10193000406FF3503F27F450402303E23F374035D8
:10194000D8B0E8682D6F1200080EF326060EF422B8
:101950000ED0080EF326090EF42209D0080EF32645
:101960000C0EF42204D0080EF3260F0EF422F3CF4F
:10197000F6FFF4CFF7FFF86A0900F5CF3DF1090053
:10198000F5CF3EF10900F5CF3FF1C2D74CC120F0B1
:1019900001011C9A4A5109E0E84C14D0E84C25D0CA
:1019A000E84C4AD0E84C4FD059D08982929276ECDC
:1019B0000DF01C961C981D901D981D9A2BC04FF180
:1019C0004A2B010C1D921D98495106E04F512B5C8A
:1019D0001408D8B0D10C07D01C984F512B5C0508C7
:1019E000D8B0D20C00D04A2B020C3BC2E8FFF20860
:1019F000D8A0030C3DC2E8FF485DD8B0040C1DB66A
:101A000003D0800E326F0AD01DA2050C32C13AF10C
:101A100006801DA403D0800E326F1D9689921D9200
:101A200092821C861C8C010E306F6A6AC00E6B1687
:101A30004A2B2BC04FF1060C4F512B5C0208D8B03B
:101A4000D30C4A2B070C39C2E8FFF208D8A0080CC7
:101A50003F0E6B121D92496B4A2B090C1DA214D02C
:101A60001DB609D01D861D923AC132F10DD01D96CA
:101A7000800E326F09D01D9232C13AF106801DB43A
:101A8000F6D71C961D98316B1D8A1DB81C961CA696
:101A900006D032C131F106A639C131F101D0316B26
:101AA0003051316333D0D8A42CD01DB024D01DB810
:101AB00022D01CBC1BD01CB6100C1D9A898292929D
:101AC0002BC04FF1496B010E4A6F110C8982929223
:101AD0001D861C961D901D981D9AE84AE868E8CF5F
:101AE00049F1E86AE8CF4AF1A00E03261C9C6A6A15
:101AF000C00E6B16120C1C781D9832C131F11C8679
:101B0000130C1DA0140C1C96316B150C3051D8A46D
:101B100005D01CBC03D01C8C3F0E6B12316503D06A
:101B2000304B3069160C3007D8A0306B170C150CF1
:101B300001015BB13BD02E4B2F2B5B8150C156F185
:101B400051C157F152C158F15351565F5451575B2F
:101B50005551585B50C153F151C154F152C155F127
:101B6000020116C21CF217C21DF218C21EF219C2DF
:101B70001FF21AC220F21BC221F226C22CF227C287
:101B80002DF228C22EF229C22FF22AC230F22BC225
:101B900031F2166B176B186B196B1A6B1B6B26697E
:101BA0002769286929692A692B6912001200010135
:101BB000A68E18C11BF119C11CF11AC11DF118C163
:101BC0001EF119C11FF11AC120F11CA80DD0550E2C
:101BD0001B27550E1C23550E1D23AA0E1E27AA0EC9
:101BE0001F23AA0E20230CD0AA0E1B27AA0E1C23EB
:101BF000AA0E1D23550E1E27550E1F23550E2023FA
:101C00001DC1F6FFF76AF636F736F690F86A080E49
:101C1000F626020EF722000EF8220900F5502D03D9
:101C2000F3CF21F1F4CF22F1236B0900F5502D03FE
:101C3000F3502227F4502323F5AE02D02D51235F19
:101C4000010E21277F0E22237F0E2323990E225F70
:101C5000190E235B21E3CC0E225DCC0E235917E233
:101C600023514203F4CF28F1F3CF27F12251256B02
:101C70004203F4502727E86A2823266FF4502727C9
:101C8000E86A282327C177FF28C176FF07D0FE0E18
:101C9000776E3F0E766E02D0776A766A20C1F6FFC5
:101CA000F76AF636F736F690F86A080EF626020E50
:101CB000F722000EF8220900F5502D03F3CF21F191
:101CC000F4CF22F1236B0900F5502D03F3502227A6
:101CD000F4502323F5AE02D02D51235F010E2127AE
:101CE0007F0E22237F0E2323990E225F190E235B82
:101CF00021E3CC0E225DCC0E235917E2235142037F
:101D0000F4CF28F1F3CF27F12251256B4203F45091
:101D10002727E86A2823266FF4502727E86A282314
:101D200027C175FF28C174FF07D0FE0E756E3F0EE8
:101D3000746E02D0756A746A1AC1F6FFF76AF636D5
:101D4000F736F690F86A080EF626020EF722000E15
:101D5000F8220900F5502D03F3CF21F1F4CF22F141
:101D6000236B0900F5502D03F3502227F450232351
:101D7000F5AE02D02D51235F010E21277F0E2223C5
:101D80007F0E2323990E225F190E235B21E3CC0ED5
:101D9000225DCC0E235917E223514203F4CF28F1E0
:101DA000F3CF27F12251256B4203F4502727E86A2D
:101DB0002823266FF4502727E86A282327C179FFB4
:101DC00028C178FF07D0FE0E796E3F0E786E02D0E4
:101DD000796A786A1C9012001E500000E82CFDD72A
:021DE0001200EF
:0E1DE2000BEF13F04651080802E20FEF11F06C
:101DF0001E0EFA6ED8904635020FD8B0FA2AFB6A4A
:101E0000F96E0AD03CD078D0BED0FAD01CD15AD1CD
:101E100089D1B8D1E7D1010C0D0E520352BFF45E47
:101E2000F80EF326F70EF4223751F402F4CF4AF2FB
:101E3000F3CF49F23651F302F4CF4EF2F3CF47F22B
:101E4000F402F3504E27F4504923E86A4A233751ED
:101E5000F302F3504E25486FF4504923E86A4A23B1
:101E6000D8904A334933D8904A334933D8904A33CB
:101E7000493349C26BF24AC26CF2462B000C1DAAD0
:101E800008D045C1E8FF395D01E203D0050E66ECDC
:101E90000DF0820E510351BFF45E780EF3262D0E25
:101EA000F4223951F402F4CF4AF2F3CF49F2385117
:101EB000F302F4CF4EF2F3CF47F2F402F3504E2781
:101EC000F4504923E86A4A233951F302F3504E256E
:101ED000486FF4504923E86A4A23D8904A3349337B
:101EE000D8904A334933D8904A33493349C267F2CC
:101EF0004AC268F2462B000C46C1E8FF3B5D01E296
:101F000003D0060E66EC0DF0820E500350BFF45E57
:101F1000800EF3263F0EF4223B51F402F4CF4AF236
:101F2000F3CF49F23A51F302F4CF4EF2F3CF47F236
:101F3000F402F3504E27F4504923E86A4A233B51F8
:101F4000F302F3504E25486FF4504923E86A4A23C0
:101F5000D8904A334933D8904A334933D8904A33DA
:101F60004933D8904A334933D8904A334933D890CB
:101F70004A334933D8904A33493349C269F24AC295
:101F80006AF2462B000C47C1E8FF3D5D02E28B96EA
:101F900004D08B86070E66EC0DF0820E4F034FBF08
:101FA000F45E780EF326E60EF4223D51F402F4CFEF
:101FB0004AF2F3CF49F23C51F302F4CF4EF2F3CFA1
:101FC00047F2F402F3504E27F4504923E86A4A23BB
:101FD0003D51F302F3504E25486FF4504923E86A0F
:101FE0004A23D8904A334933D8904A334933D8905A
:101FF0004A33493349C265F24AC266F2462B000CA5
:1020000066516A03F4CF4AF2F3CF49F2655169038E
:10201000F4CF4EF2F3CF47F26A03F3504E27F45059
:102020004923E86A4A2366516903F3504E25486FF5
:10203000F4504923E86A4A2348C271F249C272F255
:1020400018921896000C0D0E530353BFF45E800EC9
:10205000F326CF0EF4223F51F402F4CF4AF2F3CF2D
:1020600049F23E51F302F4CF4EF2F3CF47F2F402BD
:10207000F3504E27F4504923E86A4A233F51F302B4
:10208000F3504E25486FF4504923E86A4A23D8900C
:102090004A334933D8904A334933D8904A33493385
:1020A000D8904A334933D8904A334933D8904A3389
:1020B0004933D8904A33493349C26DF24AC26EF26D
:1020C000462B000C0D0E540354BFF45E800EF32615
:1020D000CF0EF4223751F402F4CF4AF2F3CF49F293
:1020E0003651F302F4CF4EF2F3CF47F2F402F3503D
:1020F0004E27F4504923E86A4A233751F302F3503C
:102100004E25486FF4504923E86A4A23D89048374F
:1021100049374A37010E4A1749C26DF24AC26EF278
:10212000462B000C0D0E550355BFF45E800EF326B2
:10213000CF0EF4223F51F402F4CF4AF2F3CF49F22A
:102140003E51F302F4CF4EF2F3CF47F2F402F350D4
:102150004E27F4504923E86A4A233F51F302F350D3
:102160004E25486FF4504923E86A4A23D8904837EF
:1021700049374A37010E4A1749C26DF24AC26EF218
:10218000462B000C0D0E560356BFF45E800EF32650
:10219000CF0EF4223F51F402F4CF4AF2F3CF49F2CA
:1021A0003E51F302F4CF4EF2F3CF47F2F402F35074
:1021B0004E27F4504923E86A4A233F51F302F35073
:1021C0004E25486FF4504923E86A4A23D89048378F
:1021D00049374A37010E4A1749C26FF24AC270F2B4
:1021E000462B000C18941896000C462B000C1894E3
:1021F0001896000C000C020118B6F5D518B204D0E0
:1022000018B407D018901200000E466F1886F0D54B
:102210001200050E466F1886EBD5120012001890BA
:0C2220001892189418961A6A466B120067
:04222C000BEF13F0B1
:10223000330C98229E22B422CA22D722DF22E72220
:102240000F234A2352235C2371238723902399234E
:10225000A223AB23B423BD23C623CF23D923F22348
:102260000B2424243E244F2460247A249424AE2476
:10227000C824E224FA2412252A2542255A25742549
:1022800074257425742574258E25A125B425C825AB
:10229000DC25F525F525F52500280C06010014534D
:1022A00074617274205445535420526967687420D5
:1022B0004B65790014436F6E74696E75652D4D69B9
:1022C00064646C65204B657920001F1226003A1269
:1022D00025003A12240000001600FF1613FF00002C
:1022E0001600201613200027182C001A6100164033
:1022F0001030012C102D012C104A012C1049011016
:102300004B011A79000000000000000000000027C7
:10231000182C0016481967021647543D1614104928
:1023200001101900104B011653196502562C165A4C
:10233000196902412C13710216675716071A3401E6
:102340001A3601001627182C00000020134D01201A
:102350000000003D3D3D3D3D3D3D00000016004676
:102360006F72773E3E3E160D3D1032012053706471
:102370000000160020537064201032013D160E3C00
:102380003C3C526576001A003D53544F503D3D0091
:102390000052554E2020202000002052554E202073
:1023A000200000202052554E2020000020202052E6
:1023B000554E2000002020202052554E00002020A5
:1023C0002052554E200000202052554E2020000063
:1023D0002052554E202020000001121600202053CC
:1023E00070656564204D6F746F723D170CFF103976
:1023F000010001121600202020202020562F462008
:10240000416D703D1700FF104301000112160020BE
:10241000202020562F462053746172743D1700FF10
:102420001044010001121600202020416363656CF6
:1024300065726174653D1701FF104C0100000112C7
:10244000160057312054656D7020466C743D0001B4
:10245000121600573120546D703120466C743D00C7
:10246000011216005465726D697374204661756CB3
:10247000743D1700FF1045010000011216004F7651
:10248000657243757272656E7420413D1700FF10CE
:1024900046010000011216004F766572566F6C748B
:1024A00061676520563D1700FF10470100000112CB
:1024B000160020556E646572566F6C742055563D3B
:1024C0001700FF1048010000011216004D4158206E
:1024D00053706420496E6465783D1700FF103C011D
:1024E00000000112160020202034363056204164AE
:1024F0006A3D170000144F02000001121600202050
:10250000374120312041646A3D20170000145002F9
:102510000000011216005465726D697374204164E5
:102520006A3D17000014510200000112160020201D
:1025300032354120332041646A3D170000145202B5
:102540000000011216002056617269616E74203419
:10255000733D172B301479000000011216004465FA
:10256000626F756E63652054696D653D172B301081
:10257000810000000112160020202044656C617962
:1025800020546573743D1701FF101E00000054169F
:1025900054313D196502562C196902412C10140062
:1025A00000541654323D196702432C196B02412C1A
:1025B00010140000541654333D196902562C196D3D
:1025C0000241002C00000000541654343D196B02E7
:1025D000562C196F0241002C0000000054165411B3
:1025E00036024D3D111C02202045101900101F001D
:1025F0002010140000541654353D103702103902D3
:10260000103B02103D02103F021041021043021025
:062610004502202000003D
:0A261600700ED36E89829292D0CF2D
:1026200060F0D08ED098D082D0800001C00E936E22
:10263000000E946E000E956EFC6A22EEFFF0000113
:10264000730ED36E94969494F86A9598036AD0A604
:1026500003060001959E959C959A8C9E8C9C8C9A65
:10266000046A056A066A076A046A146A166A176ABF
:102670000686050E616F0201C26AC280C288C28AE4
:10268000C284C16AC188C06AC082C08CC08E9A6A86
:102690009A8EB868B96892689668B898996AC28044
:1026A0009F9C9E9C9D8CC282200E016F400E026FEB
:1026B000196A036B046B056B066B076B086B096B80
:1026C0000A6B0B6B0C6B0D6B0E6B0F6B106B116B46
:1026D0000101786A1F0E796E766A1F0E776E746A32
:1026E0001F0E756E040E7A6E040E7B6E7F6A7F82FB
:1026F0007F807E6A7E8E6F6A6F8C6E6A6D6A180E3E
:102700006D6E6B686A6A6C6A150E396F850E436F61
:102710001F6A01011D6A1C6A4A6B496B2E6B2F6B85
:10272000336B0D0E346F080E356F0A0E366F000EC8
:10273000416F140E426F316B1C9676EC0DF0A5982C
:10274000A498A398D0B603D01D86010E496FF29EBF
:10275000F29C6AEC14F00101246A256A266A276A51
:102760002C6A140E5F6FBC0E606F540E616F080E02
:10277000626F91689068886A876AB76AB78CB78019
:10278000A580A490A380F28EF28CD180016A026AA7
:1027900006D0014E029402B009D0025007E11E0E8D
:1027A0001B6E020E016E028002840400000105A867
:1027B00004EC09F000B2C2EC0BF000B4BEEC0BF07C
:1027C00000B6F6EC0BF018B0FBEC10F01CB260ECAD
:1027D0000CF01CAA03D0C6EC0CF04B6F1CBE98EC9E
:1027E0000DF006B028EC14F00201133F04D0143FA2
:1027F00002D0143F00D0010100B085EC14F0C9D71D
:10280000D890E846E846E890FD26000EFE22120029
:102810000BEF13F0450146014701480139013A0128
:102820003B013C01430144011E004C0179004F0271
:1028300050025102520253025402550256025702EC
:102840008100580259025A025B025C025D025E027C
:102850000101A6B21200A694A19806B206D05C6B44
:10286000140E5D6F280E5E6F0682A69CF86A5DC12D
:10287000F6FF5EC1F7FFA68E0900F5CFE9FF09005C
:10288000F5CFEAFFF6CF5DF1F7CF5EF1EA6604D04F
:10289000E96602D0F1D71200F29CA69E5CC1A9FFA6
:1028A000A680EF50A8620AD8A68EF28C5C2B1E0E72
:1028B0005C6101D01200069006921200A86E232AD5
:1028C000A684F29E550EA76EAA0EA76EA682A694A7
:1028D000F28E120001015C6BA69C140EF66E280E9F
:1028E000F76EF86AA68E0900F5CFE9FF0900F5CF6B
:1028F000EAFFA69E5CC1A9FFA6800000A850EF6E6B
:0A2900005C2B1E0E5C611200EDD787
:06290A00060E06B6E828E7
:102910000C6E0598078206A602D015BA176A020146
:10292000F29E13C282F014C283F015C284F0136BBE
:10293000146B156BF28E01011C741CB408D00101DC
:10294000090E1CBC0C0E1CA601D0080E346F080E1C
:102950001CA6E828356F0A0E1CB8E828366F01015E
:1029600000902C2A020E2C5CD8A400D0090E2C64F6
:1029700012000101F29E2EC137F12FC138F12E6BEA
:102980002F6BF28E37513C0DF3CF21F1F4CF22F1B2
:1029900038513C0DF350222721C14DF122C14EF197
:1029A000010104B0176A172A06B602D00C0E01D036
:1029B000030E176404D00676176A056A076A2C6A44
:1029C000242A2D2A3B0E246410D0246A252A3B0E8B
:1029D00025640BD0256A262A170E266406D0266A9F
:1029E000272A630E276401D0276A030E0B6E059811
:0429F000078012004A
:020000040030CA
:01000100C638
:010002000BF2
:0100030020DC
:0100040020DB
:010005009862
:0100060001F8
:0200000400F00A
:10000000D7CAE0A0A040C000A02301402B181920AF
:0D0010002122232425260A28292A2B2C2D05
:00000001FF
